:020000040000FA
:040000008FEF00F08E
:020008009ED088
:08001800ECD00B6E960E036E96
:10002000980E046E55D8D8B4CA90D8A4CA80FC0FD4
:10003000D8A0CA92D8B0CA82800E036E960E046E03
:10004000980E076E086ACAB025D8CAB223D842D81B
:100050000304CB6E03C005F004C006F00050096E27
:100060000A6E003C0A6A4BD808500B2E0AD0BE6EAE
:100070000C0EBD6E07BEBD8A07BCBD889394CA84B2
:100080001200BB6E0C0EBA6E07BEBA8A07BCBA88E5
:100090009492F5D700D8D890073204320332120078
:1000A000066A056EFF0E0526062200D0D8A01200B3
:1000B000030E046EE70E02D8F5D7046AFE0F036E36
:1000C000E86A045AD8A012000000030600D0F8D74E
:1000D000086A076A100EF36E0434073608360550B6
:1000E000075C0650085805E30550075E0650085A9D
:1000F000D88003360436F32EEFD703501200055094
:100100000902F3CF07F0F4CF08F006500902F350CC
:10011000082605500A02F350082607501200F86A14
:100120004F0EAF6E240EAC6E900EAB6E0001C69AF1
:10013000400E926EE00E936EC00E946E070EB46E7B
:100140000F0EC16E9DD09EAA1BD0060EAB1412E1FD
:10015000E1CF3FF0E2CF40F0412A1EEE80F0415067
:10016000E126000EE222AECFE7FF3FC0E1FF40C034
:10017000E2FF1100AE50AE50AB98AB8811000AD030
:10018000F2A408D0F2940E4A0F2A817A0D6AD6CFD3
:100190000CF0110011004150425C14E0422AE9CFFA
:1001A00003F0EACF04F00EEE80F04250E926000E94
:1001B000EA22EF50036E03C0E9FF04C0EAFFD880D3
:1001C000120004D0E868036ED8A012001200416A41
:1001D000426A9D8A9F8AF28EF28C12009D9A0EEEE0
:1001E00080F0000EEE6AE82EFDD7416A426A9D8AD1
:1001F0001200F29ED8CF5AFEE8CF5BFEE0CF5CFE45
:10020000E9CF5DFEEACF5EFEE1CF5FFEE2CF60FEAA
:10021000D9CF61FEDACF62FEF6CF63FEF7CF64FE80
:10022000F5CF65FEF3CF66FEF4CF67FEA6CF68FE7E
:10023000F28E0001A192F29E5ACED8FF5BCEE8FF6B
:100240005CCEE0FF5DCEE9FF5ECEEAFF5FCEE1FF70
:1002500060CEE2FF61CED9FF62CEDAFF63CEF6FF59
:1002600064CEF7FF65CEF5FF66CEF3FF67CEF4FFF1
:1002700068CEA6FFF28E10009EA8FED7AD6E1200CB
:1002800093948A949290899092928992929489946C
:100290009296899692988998929A899A94908B903E
:1002A00094928B9294968B9694988B98949A8B9A1E
:1002B000006A280E056E260E066E010EAEDE939ABB
:1002C0008A9A286A296A2A6A2B6A2C6A2D6A2E6AF7
:1002D0002F6A306A316A326A336A346A356A366A3A
:1002E000376A386A396A3A6A3B6A3C6A3D6A226A06
:1002F00094EC0BF091EC0DF0939A8A8A320ED0DEDA
:10030000939A8A9A206A216A266A276A60DF66DFE2
:10031000CD6AF294F28A870ED56EB16AA192A0825C
:10032000D08EA292B00EB16E36DF106EBE0E105C93
:1003300009E3FE0E105C03E31BEF05F003D0126A25
:100340001BEF05F010AE22D0126A8D0E105C05E195
:1003500010C012F01368146817D09D0E105C05E1F0
:1003600010C012F0156816680FD0AD0E105C05E1D4
:1003700010C012F01768186807D0BD0E105C04E1B9
:1003800010C012F019681A681BEF05F0125204E150
:100390001BEF05F01BEF05F08D0E125CD8A461D0A9
:1003A000132803E110C013F058D0520E135C04E17F
:1003B00020908990269050D0530E135C04E1209237
:1003C0008992269249D0540E135C04E120948994BA
:1003D000269442D0560E135C04E120968996269608
:1003E0003BD05A0E135C04E120988998269834D0AB
:1003F0005B0E135C04E1209A899A269A2DD05C0E3C
:10040000135C04E1209C8B90269C26D05D0E135C2F
:1004100004E1209E8B92269E1FD0780E135C08E18B
:10042000006A280E056E260E066E010EF6DD14D04B
:100430005E0E135C04E121928B9627920DD05F0E25
:10044000135C04E121948B98279406D0600E135C12
:1004500003E121968B9A279613681BEF05F01BEF9B
:1004600005F09D0E125CD8A401EF05F0152804E1FB
:1004700010C015F0FFEF04F010C016F01652D8A40B
:100480005BD0520E155C04E120902690899051D0EB
:10049000530E155C04E12092899226924AD0540EA4
:1004A000155C04E120948994269443D0560E155C83
:1004B00004E12096899626963CD05A0E155C04E1FC
:1004C00020988998269835D05B0E155C04E1209A17
:1004D000899A269A2ED05C0E155C04E1209C8B90A4
:1004E000269C27D05D0E155C04E1209E8B92269EF3
:1004F00020D0780E155C09E1006A280E056E260EE4
:10050000066E010E0DEC00F014D05E0E155C04E1D9
:1005100021928B9627920DD05F0E155C04E12194F9
:100520008B98279406D0600E155C03E121968B9A78
:10053000279615681BEF05F0520E155C34E1285222
:1005400002E12952D8A426802080D6CF0CF0D7CF44
:100550000DF001EEBBF0D8901634E926000EEA2229
:10056000EECF01F0EFCF02F001C043F002C044F043
:1005700043C001F044C002F001500C241C6E025034
:100580000D201D6E000E0E201E6E000E0F201F6E21
:100590001EC05BF01FC05CF01CC073F01DC074F087
:1005A0008980FEEF04F0530E155C33E12A5202E11C
:1005B0002B52D8A426822082D6CF0CF0D7CF0DF0B4
:1005C00002EEBBF0D8901634E926000EEA22EECFF8
:1005D00001F0EFCF02F001C045F002C046F045C087
:1005E00001F046C002F001500C241C6E02500D2098
:1005F0001D6E000E0E201E6E000E0F201F6E1EC000
:100600005DF01FC05EF01CC075F01DC076F08982E1
:10061000F5D1540E155C33E12C5202E12D52D8A4D1
:1006200026842084D6CF0CF0D7CF0DF003EEBBF09C
:10063000D8901634E926000EEA22EECF01F0EFCF73
:1006400002F001C047F002C048F047C001F048C0C6
:1006500002F001500C241C6E02500D201D6E000E85
:100660000E201E6E000E0F201F6E1EC05FF01FC0FA
:1006700060F01CC077F01DC078F08984BFD1560EA1
:10068000155C33E12E5202E12F52D8A42686208633
:10069000D6CF0CF0D7CF0DF004EEBBF0D8901634C7
:1006A000E926000EEA22EECF01F0EFCF02F001C002
:1006B00049F002C04AF049C001F04AC002F00150BE
:1006C0000C241C6E02500D201D6E000E0E201E6E9E
:1006D000000E0F201F6E1EC061F01FC062F01CC014
:1006E00079F01DC07AF0898689D15A0E155C33E104
:1006F000305202E13152D8A426882088D6CF0CF09F
:10070000D7CF0DF005EEBBF0D8901634E926000ED9
:10071000EA22EECF01F0EFCF02F001C04BF002C0B1
:100720004CF04BC001F04CC002F001500C241C6E88
:1007300002500D201D6E000E0E201E6E000E0F20AA
:100740001F6E1EC063F01FC064F01CC07BF01DC094
:100750007CF0898853D15B0E155C33E1325202E1A3
:100760003352D8A4268A208AD6CF0CF0D7CF0DF0EA
:1007700006EEBBF0D8901634E926000EEA22EECF42
:1007800001F0EFCF02F001C04DF002C04EF04DC0BD
:1007900001F04EC002F001500C241C6E02500D20DE
:1007A0001D6E000E0E201E6E000E0F201F6E1EC04E
:1007B00065F01FC066F01CC07DF01DC07EF0898A08
:1007C0001DD15C0E155C33E1345202E13552D8A4E0
:1007D000268C208CD6CF0CF0D7CF0DF007EEBBF0D7
:1007E000D8901634E926000EEA22EECF01F0EFCFC2
:1007F00002F001C04FF002C050F04FC001F050C0F5
:1008000002F001500C241C6E02500D201D6E000ED3
:100810000E201E6E000E0F201F6E1EC067F01FC040
:1008200068F01CC07FF01DC080F08B80E7D05D0EAB
:10083000155C33E1365202E13752D8A4268E208E61
:10084000D6CF0CF0D7CF0DF008EEBBF0D890163411
:10085000E926000EEA22EECF01F0EFCF02F001C050
:1008600051F002C052F051C001F052C002F00150EC
:100870000C241C6E02500D201D6E000E0E201E6EEC
:10088000000E0F201F6E1EC069F01FC06AF01CC052
:1008900081F01DC082F08B82B1D0780E155C0DE125
:1008A000D89016343E6E3EC000F0280E056E260E1F
:1008B000066E010E0DEC00F0A1D05E0E155C33E16A
:1008C000385202E13952D8A427822182D6CF0CF0C7
:1008D000D7CF0DF009EEBBF0D8901634E926000E04
:1008E000EA22EECF01F0EFCF02F001C055F002C0D6
:1008F00056F055C001F056C002F001500C241C6E99
:1009000002500D201D6E000E0E201E6E000E0F20D8
:100910001F6E1EC06DF01FC06EF01CC085F01DC0A4
:1009200086F08B866BD05F0E155C33E13A5202E1A4
:100930003B52D8A427842184D6CF0CF0D7CF0DF01A
:100940000AEEBBF0D8901634E926000EEA22EECF6C
:1009500001F0EFCF02F001C057F002C058F057C0CD
:1009600001F058C002F001500C241C6E02500D2002
:100970001D6E000E0E201E6E000E0F201F6E1EC07C
:100980006FF01FC070F01CC087F01DC088F08B880E
:1009900035D0600E155C32E13C5202E13D52D8A4E4
:1009A00027862186D6CF0CF0D7CF0DF00BEEBBF00B
:1009B000D8901634E926000EEA22EECF01F0EFCFF0
:1009C00002F001C059F002C05AF059C001F05AC0FB
:1009D00002F001500C241C6E02500D201D6E000E02
:1009E0000E201E6E000E0F201F6E1EC071F01FC065
:1009F00072F01CC089F01DC08AF08B8A15681BD06C
:100A00001AD0AD0E125C0BE1172803E110C017F0ED
:100A100004D010C018F037EC0AF00DD00CD0BD0E89
:100A2000125C09E1192803E110C019F004D010C0CC
:100A30001AF014EC0BF020A03CD05BC01EF05CC0A0
:100A40001FF073C01CF074C01DF0D6CF0CF0D7CFD0
:100A50000DF01C500C5C1D500D581E500E581F50B0
:100A60000F580F501F18D8B0800A22E789902090A5
:100A700026A01ED0285202E1295219E0D6CF0CF050
:100A8000D7CF0DF028500C241C6E29500D201D6E60
:100A9000000E0E201E6E000E0F201F6E1EC08BF06B
:100AA0001FC08CF01CC0A3F01DC0A4F001D0269084
:100AB00037D026A034D08BC01EF08CC01FF0A3C04E
:100AC0001CF0A4C01DF0D6CF0CF0D7CF0DF01C50F9
:100AD0000C5C1D500D581E500E581F500F580F50D3
:100AE0001F18D8B0800A1AE7208043C001F044C024
:100AF00002F001500C241C6E02500D201D6E000EE1
:100B00000E201E6E000E0F201F6E1EC05BF01FC059
:100B10005CF01CC073F01DC074F0898001D0899016
:100B200020A23CD05DC01EF05EC01FF075C01CF05E
:100B300076C01DF0D6CF0CF0D7CF0DF01C500C5C5A
:100B40001D500D581E500E581F500F580F501F1893
:100B5000D8B0800A22E78992209226A21ED02A527B
:100B600002E12B5219E0D6CF0CF0D7CF0DF02A506E
:100B70000C241C6E2B500D201D6E000E0E201E6EC0
:100B8000000E0F201F6E1EC08DF01FC08EF01CC007
:100B9000A5F01DC0A6F001D0269237D026A234D0F1
:100BA0008DC01EF08EC01FF0A5C01CF0A6C01DF0A9
:100BB000D6CF0CF0D7CF0DF01C500C5C1D500D584B
:100BC0001E500E581F500F580F501F18D8B0800AD3
:100BD0001AE7208245C001F046C002F001500C2403
:100BE0001C6E02500D201D6E000E0E201E6E000E9B
:100BF0000F201F6E1EC05DF01FC05EF01CC075F0A0
:100C00001DC076F0898201D0899220A43CD05FC0BB
:100C10001EF060C01FF077C01CF078C01DF0D6CF6A
:100C20000CF0D7CF0DF01C500C5C1D500D581E5011
:100C30000E581F500F580F501F18D8B0800A22E7C7
:100C40008994209426A41ED02C5202E12D5219E042
:100C5000D6CF0CF0D7CF0DF02C500C241C6E2D509D
:100C60000D201D6E000E0E201E6E000E0F201F6E3A
:100C70001EC08FF01FC090F01CC0A7F01DC0A8F0D0
:100C800001D0269437D026A434D08FC01EF090C057
:100C90001FF0A7C01CF0A8C01DF0D6CF0CF0D7CF16
:100CA0000DF01C500C5C1D500D581E500E581F505E
:100CB0000F580F501F18D8B0800A1AE7208447C079
:100CC00001F048C002F001500C241C6E02500D20AF
:100CD0001D6E000E0E201E6E000E0F201F6E1EC019
:100CE0005FF01FC060F01CC077F01DC078F08984F1
:100CF00001D0899420A63CD061C01EF062C01FF0D4
:100D000079C01CF07AC01DF0D6CF0CF0D7CF0DF013
:100D10001C500C5C1D500D581E500E581F500F5883
:100D20000F501F18D8B0800A22E78996209626A671
:100D30001ED02E5202E12F5219E0D6CF0CF0D7CFA1
:100D40000DF02E500C241C6E2F500D201D6E000E29
:100D50000E201E6E000E0F201F6E1EC091F01FC0D1
:100D600092F01CC0A9F01DC0AAF001D0269637D081
:100D700026A634D091C01EF092C01FF0A9C01CF06E
:100D8000AAC01DF0D6CF0CF0D7CF0DF01C500C5CD4
:100D90001D500D581E500E581F500F580F501F1841
:100DA000D8B0800A1AE7208649C001F04AC002F094
:100DB00001500C241C6E02500D201D6E000E0E20E2
:100DC0001E6E000E0F201F6E1EC061F01FC062F06D
:100DD0001CC079F01DC07AF0898601D0899620A8C0
:100DE0003CD063C01EF064C01FF07BC01CF07CC010
:100DF0001DF0D6CF0CF0D7CF0DF01C500C5C1D5061
:100E00000D581E500E581F500F580F501F18D8B0B5
:100E1000800A22E78998209826A81ED0305202E145
:100E2000315219E0D6CF0CF0D7CF0DF030500C2452
:100E30001C6E31500D201D6E000E0E201E6E000E19
:100E40000F201F6E1EC093F01FC094F01CC0ABF0AB
:100E50001DC0ACF001D0269837D026A834D093C05E
:100E60001EF094C01FF0ABC01CF0ACC01DF0D6CF7C
:100E70000CF0D7CF0DF01C500C5C1D500D581E50BF
:100E80000E581F500F580F501F18D8B0800A1AE77D
:100E900020884BC001F04CC002F001500C241C6EA5
:100EA00002500D201D6E000E0E201E6E000E0F2033
:100EB0001F6E1EC063F01FC064F01CC07BF01DC01D
:100EC0007CF0898801D0899820AA3CD065C01EF0AA
:100ED00066C01FF07DC01CF07EC01DF0D6CF0CF0A8
:100EE000D7CF0DF01C500C5C1D500D581E500E58E5
:100EF0001F500F580F501F18D8B0800A22E7899A48
:100F0000209A26AA1ED0325202E1335219E0D6CFDF
:100F10000CF0D7CF0DF032500C241C6E33500D2046
:100F20001D6E000E0E201E6E000E0F201F6E1EC0C6
:100F300095F01FC096F01CC0ADF01DC0AEF001D002
:100F4000269A37D026AA34D095C01EF096C01FF03E
:100F5000ADC01CF0AEC01DF0D6CF0CF0D7CF0DF059
:100F60001C500C5C1D500D581E500E581F500F5831
:100F70000F501F18D8B0800A1AE7208A4DC001F020
:100F80004EC002F001500C241C6E02500D201D6E4C
:100F9000000E0E201E6E000E0F201F6E1EC065F08C
:100FA0001FC066F01CC07DF01DC07EF0898A01D094
:100FB000899A20AC3CD067C01EF068C01FF07FC08B
:100FC0001CF080C01DF0D6CF0CF0D7CF0DF01C5018
:100FD0000C5C1D500D581E500E581F500F580F50CE
:100FE0001F18D8B0800A22E78B90209C26AC1ED018
:100FF000345202E1355219E0D6CF0CF0D7CF0DF0C4
:1010000034500C241C6E35500D201D6E000E0E2029
:101010001E6E000E0F201F6E1EC097F01FC098F0AE
:101020001CC0AFF01DC0B0F001D0269C37D026AC5C
:1010300034D097C01EF098C01FF0AFC01CF0B0C0F5
:101040001DF0D6CF0CF0D7CF0DF01C500C5C1D500E
:101050000D581E500E581F500F580F501F18D8B063
:10106000800A1AE7208C4FC001F050C002F00150F6
:101070000C241C6E02500D201D6E000E0E201E6EE4
:10108000000E0F201F6E1EC067F01FC068F01CC04E
:101090007FF01DC080F08B8001D08B9020AE3CD0C3
:1010A00069C01EF06AC01FF081C01CF082C01DF034
:1010B000D6CF0CF0D7CF0DF01C500C5C1D500D5846
:1010C0001E500E581F500F580F501F18D8B0800ACE
:1010D00022E78B92209E26AE1ED0365202E1375276
:1010E00019E0D6CF0CF0D7CF0DF036500C241C6E83
:1010F00037500D201D6E000E0E201E6E000E0F20AC
:101100001F6E1EC099F01FC09AF01CC0B1F01DC028
:10111000B2F001D0269E37D026AE34D099C01EF052
:101120009AC01FF0B1C01CF0B2C01DF0D6CF0CF0B9
:10113000D7CF0DF01C500C5C1D500D581E500E5892
:101140001F500F580F501F18D8B0800A1AE7208E72
:1011500051C001F052C002F001500C241C6E02502C
:101160000D201D6E000E0E201E6E000E0F201F6E35
:101170001EC069F01FC06AF01CC081F01DC082F063
:101180008B8201D08B9221A23CD06DC01EF06EC02C
:101190001FF085C01CF086C01DF0D6CF0CF0D7CF55
:1011A0000DF01C500C5C1D500D581E500E581F5059
:1011B0000F580F501F18D8B0800A22E78B96219243
:1011C00027A21ED0385202E1395219E0D6CF0CF0D6
:1011D000D7CF0DF038500C241C6E39500D201D6EE9
:1011E000000E0E201E6E000E0F201F6E1EC09DF002
:1011F0001FC09EF01CC0B5F01DC0B6F001D02792F4
:1012000037D027A234D09DC01EF09EC01FF0B5C0BD
:101210001CF0B6C01DF0D6CF0CF0D7CF0DF01C508F
:101220000C5C1D500D581E500E581F500F580F507B
:101230001F18D8B0800A1AE7218255C001F056C0A5
:1012400002F001500C241C6E02500D201D6E000E89
:101250000E201E6E000E0F201F6E1EC06DF01FC0F0
:101260006EF01CC085F01DC086F08B8601D08B9679
:1012700021A43CD06FC01EF070C01FF087C01CF0CE
:1012800088C01DF0D6CF0CF0D7CF0DF01C500C5CF1
:101290001D500D581E500E581F500F580F501F183C
:1012A000D8B0800A22E78B98219427A41ED03A5206
:1012B00002E13B5219E0D6CF0CF0D7CF0DF03A50F7
:1012C0000C241C6E3B500D201D6E000E0E201E6E59
:1012D000000E0F201F6E1EC09FF01FC0A0F01CC08C
:1012E000B7F01DC0B8F001D0279437D027A434D070
:1012F0009FC01EF0A0C01FF0B7C01CF0B8C01DF00A
:10130000D6CF0CF0D7CF0DF01C500C5C1D500D58F3
:101310001E500E581F500F580F501F18D8B0800A7B
:101320001AE7218457C001F058C002F001500C2484
:101330001C6E02500D201D6E000E0E201E6E000E43
:101340000F201F6E1EC06FF01FC070F01CC087F012
:101350001DC088F08B8801D08B9821A63CD071C02D
:101360001EF072C01FF089C01CF08AC01DF0D6CFDD
:101370000CF0D7CF0DF01C500C5C1D500D581E50BA
:101380000E581F500F580F501F18D8B0800A22E770
:101390008B9A219627A61ED03C5202E13D5219E0BD
:1013A000D6CF0CF0D7CF0DF03C500C241C6E3D5026
:1013B0000D201D6E000E0E201E6E000E0F201F6EE3
:1013C0001EC0A1F01FC0A2F01CC0B9F01DC0BAF031
:1013D00001D0279637D027A634D0A1C01EF0A2C0D6
:1013E0001FF0B9C01CF0BAC01DF0D6CF0CF0D7CF9B
:1013F0000DF01C500C5C1D500D581E500E581F5007
:101400000F580F501F18D8B0800A1AE7218659C00C
:1014100001F05AC002F001500C241C6E02500D2045
:101420001D6E000E0E201E6E000E0F201F6E1EC0C1
:1014300071F01FC072F01CC089F01DC08AF08B8A49
:1014400001D08B9A26502024016E27502120026E55
:1014500001100BE1010E0F5C08E30E6A0F6A896A46
:101460008B908B928B968B988B9A94EF01F0520E07
:10147000175C11E118520CE000EEBBF0D890183464
:10148000E926000EEA22EECF28F0EFCF29F002D0B5
:10149000286A296AC7D0530E175C11E118520CE074
:1014A00000EEBBF0D8901834E926000EEA22EECF09
:1014B0002AF0EFCF2BF002D02A6A2B6AB3D0540E59
:1014C000175C11E118520CE000EEBBF0D890183414
:1014D000E926000EEA22EECF2CF0EFCF2DF002D05D
:1014E0002C6A2D6A9FD0560E175C11E118520CE041
:1014F00000EEBBF0D8901834E926000EEA22EECFB9
:101500002EF0EFCF2FF002D02E6A2F6A8BD05A0E1A
:10151000175C11E118520CE000EEBBF0D8901834C3
:10152000E926000EEA22EECF30F0EFCF31F002D004
:10153000306A316A77D05B0E175C11E118520CE00B
:1015400000EEBBF0D8901834E926000EEA22EECF68
:1015500032F0EFCF33F002D0326A336A63D05C0EE0
:10156000175C11E118520CE000EEBBF0D890183473
:10157000E926000EEA22EECF34F0EFCF35F002D0AC
:10158000346A356A4FD05D0E175C11E118520CE0D9
:1015900000EEBBF0D8901834E926000EEA22EECF18
:1015A00036F0EFCF37F002D0366A376A3BD05E0EA6
:1015B000175C11E118520CE000EEBBF0D890183423
:1015C000E926000EEA22EECF38F0EFCF39F002D054
:1015D000386A396A27D05F0E175C11E118520CE0A7
:1015E00000EEBBF0D8901834E926000EEA22EECFC8
:1015F0003AF0EFCF3BF002D03A6A3B6A13D0600E6C
:10160000175C10E118520CE000EEBBF0D8901834D3
:10161000E926000EEA22EECF3CF0EFCF3DF002D0FB
:101620003C6A3D6A17681200420E195C07E11A52C3
:1016300002E121D802D08A84226804D07B0E195C92
:10164000D8B402D819681200206A216A266A276A6B
:1016500089908992899489968998899A8B908B929E
:101660008B968B988B9A006A280E056E260E066E56
:10167000010E0DEF00F0206A216A266A276A8A941B
:1016800089908992899489968998899A8B908B926E
:101690008B968B988B9A286A296A2A6A2B6A2C6AFD
:1016A0002D6A2E6A2F6A306A316A326A336A346A66
:1016B000356A366A376A386A396A3A6A3B6A3C6A16
:1016C0003D6A006A280E056E260E066E010E0DECB0
:1016D00000F0226A1200CBEC00F0106EBE0E105C1F
:1016E00004E3FE0E105C01E2126A10AE09D0126A29
:1016F000BD0E105C04E110C012F019681A6813D016
:10170000BD0E125C10E1192803E110C019F00BD0D6
:1017100010C01AF01A5207E0420E195C04E18A84E4
:10172000226894EF01F0D7D7C30EBD6FA20EBE6F33
:10173000990EBF6F980EC06FC20EC16F930EC26F2D
:10174000120EC36F8F0EC46F880EC56F8A0EC66FE0
:10175000230EC76F860EC86FE10EC96F810ECA6F68
:10176000C30ECB6F7D0ECC6FC50ECD6F790ECE6FD5
:10177000E80ECF6F750ED06F2B0ED16F720ED26F39
:101780008B0ED36F6E0ED46F0A0ED56F6B0ED66FA5
:10179000A40ED76F670ED86F5B0ED96F640EDA6F29
:1017A0002C0EDB6F610EDC6F160EDD6F5E0EDE6FD2
:1017B0001A0EDF6F5B0EE06F360EE16F580EE26FB0
:1017C0006A0EE36F550EE46FB40EE56F520EE66FCE
:1017D000150EE76F500EE86F8A0EE96F4D0EEA6F37
:1017E000140EEB6F4B0EEC6FB30EED6F480EEE6FF9
:1017F000640EEF6F460EF06F290EF16F440EF26F1C
:10180000F369410EF46FE70EF56F3F0EF66FE00ED1
:10181000F76F3D0EF86FEA0EF96F3B0EFA6F030E8D
:10182000FB6F3A0EFC6F2C0EFD6F380EFE6F640ED0
:10183000FF6F360E0101006FAA0E016F340E026FAA
:10184000FE0E036F320E046F600E056F310E066FD1
:10185000CF0E076F2F0E086F4B0E096F2E0E0A6FFB
:10186000D30E0B6F2C0E0C6F670E0D6F2B0E0E6FC1
:10187000060E0F6F2A0E106FB10E116F280E126F29
:10188000660E136F270E146F260E156F166FF10E6E
:10189000176F240E186FC50E196F230E1A6FA20E44
:1018A0001B6F220E1C6F890E1D6F210E1E6F790E8D
:1018B0001F6F200E206F710E216F1F0E226F710E91
:1018C000236F1E0E246F7A0E256F1D0E266F8B0E52
:1018D000276F1C0E286FA30E296F1B0E2A6FC30ED5
:1018E0002B6F1A0E2C6FE90E2D6F190E2E6F170E1F
:1018F0002F6F190E306F4B0E316F180E326F860E30
:10190000336F170E346FC70E356F160E366F0E0E0F
:10191000376F160E386F5B0E396F150E3A6FAD0EBE
:101920003B6F140E3C6F050E3D6F140E3E6F630E41
:101930003F6F130E406FC50E416F120E426F2D0E9A
:10194000436F120E446F990E456F110E466F0A0ECB
:10195000476F110E486F800E496F100E4A6FFA0ED6
:101960004B6F0F0E4C6F780E4D6F0F0E4E6FFA0EC1
:101970004F6F0E0E506F810E516F0E0E526F0B0E89
:10198000536F0E0E546F990E556F0D0E566F2B0E32
:10199000576F0D0E586FC00E596F0C0E5A6F580EC0
:1019A0005B6F0C0E5C6FF40E5D6F0B0E5E6F930E33
:1019B0005F6F0B0E606F350E616F0B0E626FDA0E8C
:1019C000636F0A0E646F820E656F0A0E666F2C0ECF
:1019D000676F0A0E686FDA0E696F090E6A6F8A0EFA
:1019E0006B6F090E6C6F3C0E6D6F090E6E6FF10E12
:1019F0006F6F080E706FA90E716F080E726F620E16
:101A0000736F080E746F1E0E756F080E766FDC0E06
:101A1000776F070E786F9C0E796F070E7A6F5F0EE7
:101A20007B6F070E7C6F230E7D6F070E7E6FE90EB6
:101A30007F6F060E806FB10E816F060E826F7A0E79
:101A4000836F060E846F460E856F060E866F130E2B
:101A5000876F060E886FE10E896F050E8A6FB20ED2
:101A60008B6F050E8C6F830E8D6F050E8E6F570E6C
:101A70008F6F050E906F2B0E916F050E926F010EFA
:101A8000936F050E946FD90E956F040E966FB10E7D
:101A9000976F040E986F8B0E996F040E9A6F660EF7
:101AA0009B6F040E9C6F430E9D6F040E9E6F200E65
:101AB0009F6F040EA06FFE0EA16F030EA26FDE0ECD
:101AC000A36F030EA46FBF0EA56F030EA66FA00E2B
:101AD000A76F030EA86F830EA96F030EAA6F660E81
:101AE000AB6F030EAC6F4B0EAD6F030EAE6F300ECF
:101AF000AF6F030EB06F160EB16F030EB26FFD0E17
:101B0000B36F020EB46FE50EB56F020EB66FCD0E59
:101B1000B76F020EB86FB60EB96F020EBA6F000142
:101B200012004C0E0101BD6FBE6B4E0EBF6FC06B3D
:101B3000500EC16FC26B510EC36FC46B530EC56F95
:101B4000C66B540EC76FC86B560EC96FCA6B570E63
:101B5000CB6FCC6B590ECD6FCE6B5B0ECF6FD06B56
:101B60005C0ED16FD26B5E0ED36FD46B5F0ED56FF0
:101B7000D66B610ED76FD86B630ED96FDA6B640EBC
:101B8000DB6FDC6B660EDD6FDE6B670EDF6FE06BAD
:101B9000690EE16FE26B6B0EE36FE46B6C0EE56F49
:101BA000E66B6E0EE76FE86B6F0EE96FEA6B710E16
:101BB000EB6FEC6B720EED6FEE6B740EEF6FF06B04
:101BC000760EF16FF26B770EF36FF46B790EF56FA3
:101BD000F66B7A0EF76FF86B7C0EF96FFA6B7E0E70
:101BE000FB6FFC6B7F0EFD6FFE6B810EFF6F0201C2
:101BF000006B820E016F026B840E036F046B850E07
:101C0000056F066B870E076F086B890E096F0A6BED
:101C10008A0E0B6F0C6B8C0E0D6F0E6B8D0E0F6F93
:101C2000106B8F0E116F126B910E136F146B920E5F
:101C3000156F166B940E176F186B950E196F1A6B44
:101C4000970E1B6F1C6B990E1D6F1E6B9A0E1F6FEC
:101C5000206B9C0E216F226B9D0E236F246B9F0EB9
:101C6000256F266BA00E276F286BA20E296F2A6B9B
:101C7000A40E2B6F2C6BA50E2D6F2E6BA70E2F6F46
:101C8000306BA80E316F326BAA0E336F346BAC0E13
:101C9000356F366BAD0E376F386BAF0E396F3A6BF1
:101CA000B00E3B6F3C6BB20E3D6F3E6BB30E3F6FA1
:101CB000406BB50E416F426BB70E436F446BB80E6D
:101CC000456F466BBA0E476F486BBB0E496F4A6B48
:101CD000BD0E4B6F4C6BBF0E4D6F4E6BC00E4F6FFA
:101CE000506BC20E516F526BC30E536F546BC50EC7
:101CF000556F566BC70E576F586BC80E596F5A6B9E
:101D0000CA0E5B6F5C6BCB0E5D6F5E6BCD0E5F6F53
:101D1000606BCE0E616F626BD00E636F646BD20E20
:101D2000656F666BD30E676F686BD50E696F6A6BF4
:101D3000D60E6B6F6C6BD80E6D6F6E6BDA0E6F6FAD
:101D4000706BDB0E716F726BDD0E736F746BDE0E7A
:101D5000756F766BE00E776F786BE10E796F7A6B4B
:101D6000E30E7B6F7C6BE50E7D6F7E6BE60E7F6F07
:101D7000806BE80E816F826BE90E836F846BEB0ED4
:101D8000856F866BED0E876F886BEE0E896F8A6BA1
:101D9000F00E8B6F8C6BF10E8D6F8E6BF30E8F6F61
:101DA000906BF50E916F926BF60E936F946BF80E2D
:101DB000956F966BF90E976F986BFB0E996F9A6BF8
:101DC000FC0E9B6F9C6BFE0E9D6F9E6B9F6B010EBE
:101DD000A06FA16FA26F030EA36F010EA46F040E7C
:101DE000A56F010EA66F060EA76F010EA86F080E55
:101DF000A96F010EAA6F090EAB6F010EAC6F0B0E2F
:101E0000AD6F010EAE6F0C0EAF6F010EB06F0E0E08
:101E1000B16F010EB26F0F0EB36F010EB46F110EE2
:101E2000B56F010EB66F130EB76F010EB86F140EBB
:101E3000B96F010EBA6F650EBD6FBE6B660EBF6FD8
:101E4000C06B680EC16FC26B690EC36FC46B6B0E43
:101E5000C56FC66B6C0EC76FC86B6D0EC96FCA6B52
:101E60006F0ECB6FCC6B700ECD6FCE6B710ECF6FD4
:101E7000D06B730ED16FD26B740ED36FD46B760EA2
:101E8000D56FD66B770ED76FD86B780ED96FDA6BAC
:101E90007A0EDB6FDC6B7B0EDD6FDE6B7D0EDF6F32
:101EA000E06B7E0EE16FE26B7F0EE36FE46B810E01
:101EB000E56FE66B820EE76FE86B840EE96FEA6B05
:101EC000850EEB6FEC6B860EED6FEE6B880EEF6F91
:101ED000F06B890EF16FF26B8B0EF36FF46B8C0E5F
:101EE000F56FF66B8D0EF76FF86B8F0EF96FFA6B5F
:101EF000900EFB6FFC6B920EFD6FFE6B930EFF6FEF
:101F00000301006B940E016F026B960E036F046B5E
:101F1000970E056F066B980E076F086B9A0E096F88
:101F20000A6B9B0E0B6F0C6B9D0E0D6F0E6B9E0E56
:101F30000F6F106B9F0E116F126BA10E136F146B4E
:101F4000A20E156F166BA40E176F186BA50E196FE6
:101F50001A6BA60E1B6F1C6BA80E1D6F1E6BA90EB5
:101F60001F6F206BAB0E216F226BAC0E236F246BA7
:101F7000AD0E256F266BAF0E276F286BB00E296F45
:101F80002A6BB20E2B6F2C6BB30E2D6F2E6BB40E13
:101F90002F6F306BB60E316F326BB70E336F346B01
:101FA000B90E356F366BBA0E376F386BBB0E396FA3
:101FB0003A6BBD0E3B6F3C6BBE0E3D6F3E6BBF0E72
:101FC0003F6F406BC10E416F426BC20E436F446B5B
:101FD000C40E456F466BC50E476F486BC60E496F02
:101FE0004A6BC80E4B6F4C6BC90E4D6F4E6BCB0ED0
:101FF0004F6F506BCC0E516F526BCD0E536F546BB5
:10200000CF0E556F566BD00E576F586BD20E596F5F
:102010005A6BD30E5B6F5C6BD40E5D6F5E6BD60E2E
:102020005F6F606BD70E616F626BD90E636F646B0D
:10203000DA0E656F666BDB0E676F686BDD0E696FBE
:102040006A6BDE0E6B6F6C6BE00E6D6F6E6BE10E8C
:102050006F6F706BE20E716F726BE40E736F746B67
:10206000E50E756F766BE60E776F786BE80E796F1D
:102070007A6BE90E7B6F7C6BEB0E7D6F7E6BEC0EEB
:102080007F6F806BED0E816F826BEF0E836F846BC1
:10209000F00E856F866BF20E876F886BF30E896F7B
:1020A0008A6BF40E8B6F8C6BF60E8D6F8E6BF70E4A
:1020B0008F6F906BF90E916F926BFA0E936F946B1A
:1020C000FB0E956F966BFD0E976F986BFE0E996FDA
:1020D0009A6B9B6B010E9C6F9D6F9E6F020E9F6FA4
:1020E000010EA06F040EA16F010EA26F050EA36F6B
:1020F000010EA46F070EA56F010EA66F080EA76F45
:10210000010EA86F090EA96F010EAA6F0B0EAB6F1F
:10211000010EAC6F0C0EAD6F010EAE6F0D0EAF6FFA
:10212000010EB06F0F0EB16F010EB26F100EB36FD4
:10213000010EB46F120EB56F010EB66F130EB76FAE
:10214000010EB86F140EB96F010EBA6F430EBD6F5A
:10215000BE6B440EBF6FC06B450EC16FC26B470EA6
:10216000C36FC46B480EC56FC66B490EC76FC86B93
:102170004B0EC96FCA6B4C0ECB6FCC6B4D0ECD6F37
:10218000CE6B4F0ECF6FD06B500ED16FD26B510E06
:10219000D36FD46B530ED56FD66B540ED76FD86BED
:1021A000560ED96FDA6B570EDB6FDC6B580EDD6F96
:1021B000DE6B5A0EDF6FE06B5B0EE16FE26B5C0E65
:1021C000E36FE46B5E0EE56FE66B5F0EE76FE86B47
:1021D000600EE96FEA6B620EEB6FEC6B630EED6FF6
:1021E000EE6B640EEF6FF06B660EF16FF26B670EC5
:1021F000F36FF46B680EF56FF66B6A0EF76FF86BA2
:102200006B0EF96FFA6B6D0EFB6FFC6B6E0EFD6F54
:10221000FE6B6F0EFF6F0401006B710E016F026B9E
:10222000720E036F046B730E056F066B750E076FEE
:10223000086B760E096F0A6B770E0B6F0C6B790EBD
:102240000D6F0E6B7A0E0F6F106B7B0E116F126B92
:102250007D0E136F146B7E0E156F166B800E176F4D
:10226000186B810E196F1A6B820E1B6F1C6B840E1C
:102270001D6F1E6B850E1F6F206B860E216F226BEC
:10228000880E236F246B890E256F266B8A0E276FAD
:10229000286B8C0E296F2A6B8D0E2B6F2C6B8E0E7C
:1022A0002D6F2E6B900E2F6F306B910E316F326B46
:1022B000920E336F346B940E356F366B950E376F0D
:1022C000386B970E396F3A6B980E3B6F3C6B990EDB
:1022D0003D6F3E6B9B0E3F6F406B9C0E416F426BA0
:1022E0009D0E436F446B9F0E456F466BA00E476F6C
:1022F000486BA10E496F4A6BA30E4B6F4C6BA40E3B
:102300004D6F4E6BA50E4F6F506BA70E516F526BFA
:10231000A80E536F546BA90E556F566BAB0E576FCB
:10232000586BAC0E596F5A6BAE0E5B6F5C6BAF0E99
:102330005D6F5E6BB00E5F6F606BB20E616F626B54
:10234000B30E636F646BB40E656F666BB60E676F2A
:10235000686BB70E696F6A6BB80E6B6F6C6BBA0EF9
:102360006D6F6E6BBB0E6F6F706BBC0E716F726BAF
:10237000BE0E736F746BBF0E756F766BC00E776F8A
:10238000786BC20E796F7A6BC30E7B6F7C6BC50E58
:102390007D6F7E6BC60E7F6F806BC70E816F826B09
:1023A000C90E836F846BCA0E856F866BCB0E876FE9
:1023B000886BCD0E896F8A6BCE0E8B6F8C6BCF0EB8
:1023C0008D6F8E6BD10E8F6F906BD20E916F926B63
:1023D000D30E936F946BD50E956F966BD60E976F49
:1023E000986BD80E996F9A6BD90E9B6F9C6BDA0E17
:1023F0009D6F9E6BDC0E9F6FA06BDD0EA16FA26BBD
:10240000DE0EA36FA46BE00EA56FA66BE10EA76FA7
:10241000A86BE20EA96FAA6BE40EAB6FAC6BE50E76
:10242000AD6FAE6BE60EAF6FB06BE80EB16FB26B17
:10243000E90EB36FB46BEA0EB56FB66BEC0EB76F07
:10244000B86BED0EB96FBA6B390EBD6FBE6B3B0E3C
:10245000BF6FC06B3D0EC16FC26B3F0EC36FC46BCD
:10246000420EC56FC66B440EC76FC86B460EC96F70
:10247000CA6B480ECB6FCC6B4A0ECD6FCE6B4D0E38
:10248000CF6FD06B4F0ED16FD26B510ED36FD46B19
:10249000530ED56FD66B550ED76FD86B580ED96FBC
:1024A000DA6B5A0EDB6FDC6B5C0EDD6FDE6B5E0E83
:1024B000DF6FE06B600EE16FE26B630EE36FE46B66
:1024C000650EE56FE66B670EE76FE86B690EE96F07
:1024D000EA6B6B0EEB6FEC6B6E0EED6FEE6B700ECE
:1024E000EF6FF06B720EF16FF26B740EF36FF46BB3
:1024F000760EF56FF66B790EF76FF86B7B0EF96F52
:10250000FA6B7D0EFB6FFC6B7F0EFD6FFE6B820E18
:10251000FF6F0501006B840E016F026B860E036F67
:10252000046B880E056F066B8A0E076F086B8D0EA5
:10253000096F0A6B8F0E0B6F0C6B910E0D6F0E6B8C
:10254000930E0F6F106B950E116F126B980E136F29
:10255000146B9A0E156F166B9C0E176F186B9E0EF0
:10256000196F1A6BA00E1B6F1C6BA30E1D6F1E6BD9
:10257000A50E1F6F206BA70E216F226BA90E236F74
:10258000246BAB0E256F266BAE0E276F286BB00E3B
:10259000296F2A6BB20E2B6F2C6BB40E2D6F2E6B26
:1025A000B60E2F6F306BB90E316F326BBB0E336FBF
:1025B000346BBD0E356F366BBF0E376F386BC10E87
:1025C000396F3A6BC40E3B6F3C6BC60E3D6F3E6B72
:1025D000C80E3F6F406BCA0E416F426BCC0E436F0B
:1025E000446BCF0E456F466BD10E476F486BD30ED1
:1025F000496F4A6BD50E4B6F4C6BD80E4D6F4E6BBF
:10260000DA0E4F6F506BDC0E516F526BDE0E536F54
:10261000546BE00E556F566BE30E576F586BE50E1B
:10262000596F5A6BE70E5B6F5C6BE90E5D6F5E6B0B
:10263000EB0E5F6F606BEE0E616F626BF00E636F9F
:10264000646BF20E656F666BF40E676F686BF60E67
:10265000696F6A6BF90E6B6F6C6BFB0E6D6F6E6B57
:10266000FD0E6F6F706B7169726B010E736F746F1B
:10267000040E756F010E766F060E776F010E786F80
:10268000080E796F010E7A6F0A0E7B6F010E7C6F58
:102690000C0E7D6F010E7E6F0F0E7F6F010E806F2F
:1026A000110E816F010E826F130E836F010E846F06
:1026B000150E856F010E866F170E876F010E886FDE
:1026C0001A0E896F010E8A6F1C0E8B6F010E8C6FB4
:1026D0001E0E8D6F010E8E6F200E8F6F010E906F8C
:1026E000220E916F010E926F250E936F010E946F63
:1026F000270E956F010E966F290E976F010E986F3A
:102700002B0E996F010E9A6F2E0E9B6F010E9C6F10
:10271000300E9D6F010E9E6F320E9F6F010EA06FE7
:10272000340EA16F010EA26F360EA36F010EA46FBF
:10273000390EA56F010EA66F3B0EA76F010EA86F95
:102740003D0EA96F010EAA6F3F0EAB6F010EAC6F6D
:10275000410EAD6F010EAE6F440EAF6F010EB06F44
:10276000460EB16F010EB26F480EB36F010EB46F1B
:102770004A0EB56F010EB66F4C0EB76F010EB86FF3
:102780004F0EB96F010EBA6F9B0EBD6FBE6B9D0EE3
:10279000BF6FC06B9F0EC16FC26BA00EC36FC46BC7
:1027A000A20EC56FC66BA40EC76FC86BA60EC96F0D
:1027B000CA6BA80ECB6FCC6BAA0ECD6FCE6BAB0ED7
:1027C000CF6FD06BAD0ED16FD26BAF0ED36FD46B1A
:1027D000B10ED56FD66BB30ED76FD86BB40ED96F61
:1027E000DA6BB60EDB6FDC6BB80EDD6FDE6BBA0E2C
:1027F000DF6FE06BBC0EE16FE26BBE0EE36FE46B6C
:10280000BF0EE56FE66BC10EE76FE86BC30EE96FB5
:10281000EA6BC50EEB6FEC6BC70EED6FEE6BC80E7F
:10282000EF6FF06BCA0EF16FF26BCC0EF36FF46BBF
:10283000CE0EF56FF66BD00EF76FF86BD20EF96F08
:10284000FA6BD30EFB6FFC6BD50EFD6FFE6BD70ED4
:10285000FF6F0601006BD90E016F026BDB0E036F79
:10286000046BDC0E056F066BDE0E076F086BE00E67
:10287000096F0A6BE20E0B6F0C6BE40E0D6F0E6BA3
:10288000E60E0F6F106BE70E116F126BE90E136FF0
:10289000146BEB0E156F166BED0E176F186BEF0EBA
:1028A000196F1A6BF00E1B6F1C6BF20E1D6F1E6BF7
:1028B000F40E1F6F206BF60E216F226BF80E236F44
:1028C000246BFA0E256F266BFB0E276F286BFD0E0F
:1028D000296F2A6B2B692C6B010E2D6F2E6F030E47
:1028E0002F6F010E306F040E316F010E326F060E26
:1028F000336F010E346F080E356F010E366F0A0EFE
:10290000376F010E386F0C0E396F010E3A6F0E0ED5
:102910003B6F010E3C6F0F0E3D6F010E3E6F110EAF
:102920003F6F010E406F130E416F010E426F150E87
:10293000436F010E446F170E456F010E466F180E60
:10294000476F010E486F1A0E496F010E4A6F1C0E39
:102950004B6F010E4C6F1E0E4D6F010E4E6F200E11
:102960004F6F010E506F220E516F010E526F230EEA
:10297000536F010E546F250E556F010E566F270EC3
:10298000576F010E586F290E596F010E5A6F2B0E9B
:102990005B6F010E5C6F2C0E5D6F010E5E6F2E0E75
:1029A0005F6F010E606F300E616F010E626F320E4D
:1029B000636F010E646F340E656F010E666F360E25
:1029C000676F010E686F370E696F010E6A6F390EFF
:1029D0006B6F010E6C6F3B0E6D6F010E6E6F3D0ED7
:1029E0006F6F010E706F3F0E716F010E726F400EB0
:1029F000736F010E746F420E756F010E766F440E89
:102A0000776F010E786F460E796F010E7A6F480E60
:102A10007B6F010E7C6F4A0E7D6F010E7E6F4B0E39
:102A20007F6F010E806F4D0E816F010E826F4F0E12
:102A3000836F010E846F510E856F010E866F530EEA
:102A4000876F010E886F540E896F010E8A6F560EC4
:102A50008B6F010E8C6F580E8D6F010E8E6F5A0E9C
:102A60008F6F010E906F5C0E916F010E926F5E0E74
:102A7000936F010E946F5F0E956F010E966F610E4E
:102A8000976F010E986F630E996F010E9A6F650E26
:102A90009B6F010E9C6F670E9D6F010E9E6F680EFF
:102AA0009F6F010EA06F6A0EA16F010EA26F6C0ED8
:102AB000A36F010EA46F6E0EA56F010EA66F700EB0
:102AC000A76F010EA86F720EA96F010EAA6F730E89
:102AD000AB6F010EAC6F750EAD6F010EAE6F770E62
:102AE000AF6F010EB06F790EB16F010EB26F7B0E3A
:102AF000B36F010EB46F7C0EB56F010EB66F7E0E14
:102B0000B76F010EB86F800EB96F010EBA6FAF0EBE
:102B1000BD6FBE6BB00EBF6FC06BC16FC26BB10E2D
:102B2000C36FC46BB20EC56FC66BB30EC76FC86BF5
:102B3000B40EC96FCA6BB50ECB6FCC6BB60ECD6F32
:102B4000CE6BB70ECF6FD06BB80ED16FD26BD36F89
:102B5000D46BB90ED56FD66BBA0ED76FD86BBB0ED0
:102B6000D96FDA6BBC0EDB6FDC6BBD0EDD6FDE6B1D
:102B7000BE0EDF6FE06BBF0EE16FE26BC00EE36F66
:102B8000E46BE56FE66BC10EE76FE86BC20EE96FB1
:102B9000EA6BC30EEB6FEC6BC40EED6FEE6BC50E04
:102BA000EF6FF06BC60EF16FF26BC70EF36FF46B45
:102BB000C80EF56FF66BF76FF86BC90EF96FFA6B0D
:102BC000CA0EFB6FFC6BCB0EFD6FFE6BCC0EFF6F66
:102BD0000701006BCD0E016F026BCE0E036F046B0D
:102BE000CF0E056F066BD00E076F086B096F0A6B6F
:102BF000D10E0B6F0C6BD20E0D6F0E6BD30E0F6FD1
:102C0000106BD40E116F126BD50E136F146BD60EA2
:102C1000156F166BD70E176F186BD80E196F1A6BCE
:102C20001B6F1C6BD90E1D6F1E6BDA0E1F6F206B96
:102C3000DB0E216F226BDC0E236F246BDD0E256F04
:102C4000266BDE0E276F286BDF0E296F2A6BE00ED6
:102C50002B6F2C6B2D6F2E6BE10E2F6F306BE20EF6
:102C6000316F326BE30E336F346BE40E356F366BBE
:102C7000E50E376F386BE60E396F3A6BE70E3B6F38
:102C80003C6BE80E3D6F3E6BE90E3F6F406B416F52
:102C9000426BEA0E436F446BEB0E456F466BEC0ED6
:102CA000476F486BED0E496F4A6BEE0E4B6F4C6BE6
:102CB000EF0E4D6F4E6BF00E4F6F506BF10E516F6C
:102CC000526B536F546BF20E556F566BF30E576F7A
:102CD000586BF40E596F5A6BF50E5B6F5C6BF60E0A
:102CE0005D6F5E6BF70E5F6F606BF80E616F626B0E
:102CF000F90E636F646B656F666BFA0E676F686BD6
:102D0000FB0E696F6A6BFC0E6B6F6C6BFD0E6D6F6B
:102D10006E6BFE0E6F6F706B7169726B736B010E71
:102D2000746F756F766F776F786F020E796F010E23
:102D30007A6F030E7B6F010E7C6F040E7D6F010EA8
:102D40007E6F050E7F6F010E806F060E816F010E84
:102D5000826F070E836F010E846F080E856F010E60
:102D6000866F090E876F010E886F090E896F010E3D
:102D70008A6F0A0E8B6F010E8C6F0B0E8D6F010E1A
:102D80008E6F0C0E8F6F010E906F0D0E916F010EF6
:102D9000926F0E0E936F010E946F0F0E956F010ED2
:102DA000966F100E976F010E986F110E996F010EAE
:102DB0009A6F110E9B6F010E9C6F120E9D6F010E8C
:102DC0009E6F130E9F6F010EA06F140EA16F010E68
:102DD000A26F150EA36F010EA46F160EA56F010E44
:102DE000A66F170EA76F010EA86F180EA96F010E20
:102DF000AA6F190EAB6F010EAC6F190EAD6F010EFD
:102E0000AE6F1A0EAF6F010EB06F1B0EB16F010ED9
:102E1000B26F1C0EB36F010EB46F1D0EB56F010EB5
:102E2000B66F1E0EB76F010EB86F1F0EB96F010E91
:102E3000BA6FB40EBD6FBE6BBF6FC06BB50EC16F06
:102E4000C26BC36FC46BC56FC66BB60EC76FC86B62
:102E5000C96FCA6BB70ECB6FCC6BCD6FCE6BB80E94
:102E6000CF6FD06BD16FD26BB90ED36FD46BD56FE0
:102E7000D66BBA0ED76FD86BD96FDA6BBB0EDB6F20
:102E8000DC6BDD6FDE6BDF6FE06BBC0EE16FE26B66
:102E9000E36FE46BBD0EE56FE66BE76FE86BBE0EAC
:102EA000E96FEA6BEB6FEC6BBF0EED6FEE6BEF6FE4
:102EB000F06BC00EF16FF26BF36FF46BC10EF56F38
:102EC000F66BF76FF86BC20EF96FFA6BFB6FFC6B6A
:102ED000FD6FFE6BC30EFF6F0801006B016F026B8D
:102EE000C40E036F046B056F066BC50E076F086B8E
:102EF000096F0A6BC60E0B6F0C6B0D6F0E6BC70E56
:102F00000F6F106B116F126BC80E136F146B156F70
:102F1000166B176F186BC90E196F1A6B1B6F1C6B32
:102F2000CA0E1D6F1E6B1F6F206BCB0E216F226BA5
:102F3000236F246BCC0E256F266B276F286BCD0E6D
:102F4000296F2A6B2B6F2C6BCE0E2D6F2E6B2F6F74
:102F5000306BCF0E316F326B336F346B356F366B36
:102F6000D00E376F386B396F3A6BD10E3B6F3C6BBD
:102F70003D6F3E6BD20E3F6F406B416F426BD30E85
:102F8000436F446B456F466BD40E476F486B496F78
:102F90004A6BD50E4B6F4C6B4D6F4E6B4F6F506B3A
:102FA000D60E516F526B536F546BD70E556F566BD5
:102FB000576F586BD80E596F5A6B5B6F5C6BD90E9D
:102FC0005D6F5E6B5F6F606BDA0E616F626B636F7C
:102FD000646BDB0E656F666B676F686BDC0E696F29
:102FE0006A6B6B6F6C6B6D6F6E6BDD0E6F6F706B02
:102FF000716F726BDE0E736F746B756F766BDF0EB5
:10300000776F786B796F7A6BE00E7B6F7C6B7D6F7F
:103010007E6BE10E7F6F806B816F826BE20E836F40
:10302000846B856F866B876F886BE30E896F8A6B05
:103030008B6F8C6BE40E8D6F8E6B8F6F906BE50ECC
:10304000916F926B936F946BE60E956F966B976F83
:10305000986BE70E996F9A6B9B6F9C6BE80E9D6F58
:103060009E6B9F6FA06BE90EA16FA26BA36FA46B09
:10307000A56FA66BEA0EA76FA86BA96FAA6BEB0EE4
:10308000AB6FAC6BAD6FAE6BEC0EAF6FB06BB16F87
:10309000B26BED0EB36FB46BB56FB66BEE0EB76F70
:1030A000B86BB96FBA6BAF0EBD6FBE6BB00EBF6FB2
:1030B000C06BB10EC16FC26BB20EC36FC46BB30EE7
:1030C000C56FC66BB40EC76FC86BB50EC96FCA6B40
:1030D000B60ECB6FCC6BB70ECD6FCE6BB80ECF6F7D
:1030E000D06BB90ED16FD26BBA0ED36FD46BBB0E4F
:1030F000D56FD66BBC0ED76FD86BBD0ED96FDA6BA0
:10310000BE0EDB6FDC6BBF0EDD6FDE6BC00EDF6FE4
:10311000E06BC10EE16FE26BC30EE36FE46BC40EB4
:10312000E56FE66BC50EE76FE86BC60EE96FEA6BFD
:10313000C70EEB6FEC6BC80EED6FEE6BC90EEF6F49
:10314000F06BCA0EF16FF26BCB0EF36FF46BCC0E1B
:10315000F56FF66BCD0EF76FF86BCE0EF96FFA6B5D
:10316000CF0EFB6FFC6BD00EFD6FFE6BD10EFF6FB1
:103170000901006BD20E016F026BD30E036F046B5B
:10318000D40E056F066BD50E076F086BD60E096F50
:103190000A6BD70E0B6F0C6BD80E0D6F0E6BD90E22
:1031A0000F6F106BDB0E116F126BDC0E136F146B55
:1031B000DD0E156F166BDE0E176F186BDF0E196FB5
:1031C0001A6BE00E1B6F1C6BE10E1D6F1E6BE20E87
:1031D0001F6F206BE30E216F226BE40E236F246BB5
:1031E000E50E256F266BE60E276F286BE70E296F1D
:1031F0002A6BE80E2B6F2C6BE90E2D6F2E6BEA0EEF
:103200002F6F306BEB0E316F326BEC0E336F346B14
:10321000ED0E356F366BEE0E376F386BEF0E396F84
:103220003A6BF00E3B6F3C6BF20E3D6F3E6BF30E54
:103230003F6F406BF40E416F426BF50E436F446B72
:10324000F60E456F466BF70E476F486BF80E496FE9
:103250004A6BF90E4B6F4C6BFA0E4D6F4E6BFB0EBB
:103260004F6F506BFC0E516F526BFD0E536F546BD2
:10327000FE0E556F566B5769586B596B010E5A6F9E
:103280005B6F5C6F020E5D6F010E5E6F030E5F6F12
:10329000010E606F040E616F010E626F050E636FA9
:1032A000010E646F060E656F010E666F070E676F85
:1032B000010E686F080E696F010E6A6F0A0E6B6F60
:1032C000010E6C6F0B0E6D6F010E6E6F0C0E6F6F3B
:1032D000010E706F0D0E716F010E726F0E0E736F17
:1032E000010E746F0F0E756F010E766F100E776FF3
:1032F000010E786F110E796F010E7A6F120E7B6FCF
:10330000010E7C6F130E7D6F010E7E6F140E7F6FAA
:10331000010E806F150E816F010E826F160E836F86
:10332000010E846F170E856F010E866F180E876F62
:10333000010E886F190E896F010E8A6F1A0E8B6F3E
:10334000010E8C6F1B0E8D6F010E8E6F1C0E8F6F1A
:10335000010E906F1D0E916F010E926F1E0E936FF6
:10336000010E946F1F0E956F010E966F210E976FD1
:10337000010E986F220E996F010E9A6F230E9B6FAC
:10338000010E9C6F240E9D6F010E9E6F250E9F6F88
:10339000010EA06F260EA16F010EA26F270EA36F64
:1033A000010EA46F280EA56F010EA66F290EA76F40
:1033B000010EA86F2A0EA96F010EAA6F2B0EAB6F1C
:1033C000010EAC6F2C0EAD6F010EAE6F2D0EAF6FF8
:1033D000010EB06F2E0EB16F010EB26F2F0EB36FD4
:1033E000010EB46F300EB56F010EB66F310EB76FB0
:1033F000010EB86F320EB96F010EBA6F650EBD6F58
:10340000BE6B670EBF6FC06B690EC16FC26B6B0E78
:10341000C36FC46B6C0EC56FC66B6E0EC76FC86B87
:10342000700EC96FCA6B720ECB6FCC6B740ECD6F02
:10343000CE6B760ECF6FD06B780ED16FD26B790ECC
:10344000D36FD46B7B0ED56FD66B7D0ED76FD86BD9
:103450007F0ED96FDA6B810EDB6FDC6B830EDD6F55
:10346000DE6B850EDF6FE06B860EE16FE26B880E20
:10347000E36FE46B8A0EE56FE66B8C0EE76FE86B2B
:103480008E0EE96FEA6B900EEB6FEC6B920EED6FA8
:10349000EE6B930EEF6FF06B950EF16FF26B970E74
:1034A000F36FF46B990EF56FF66B9B0EF76FF86B7D
:1034B0009D0EF96FFA6B9F0EFB6FFC6BA00EFD6FFC
:1034C000FE6BA20EFF6F0A01006BA40E016F026B70
:1034D000A60E036F046BA80E056F066BAA0E076F8E
:1034E000086BAC0E096F0A6BAD0E0B6F0C6BAF0E59
:1034F0000D6F0E6BB10E0F6F106BB30E116F126B61
:10350000B50E136F146BB70E156F166BB90E176FE0
:10351000186BBA0E196F1A6BBC0E1B6F1C6BBE0EAC
:103520001D6F1E6BC00E1F6F206BC20E216F226BB2
:10353000C40E236F246BC60E256F266BC70E276F34
:10354000286BC90E296F2A6BCB0E2B6F2C6BCD0EFF
:103550002D6F2E6BCF0E2F6F306BD10E316F326B04
:10356000D30E336F346BD40E356F366BD60E376F88
:10357000386BD80E396F3A6BDA0E3B6F3C6BDC0E52
:103580003D6F3E6BDE0E3F6F406BE00E416F426B56
:10359000E10E436F446BE30E456F466BE50E476FDC
:1035A000486BE70E496F4A6BE90E4B6F4C6BEB0EA5
:1035B0004D6F4E6BED0E4F6F506BEE0E516F526BA9
:1035C000F00E536F546BF20E556F566BF40E576F2F
:1035D000586BF60E596F5A6BF80E5B6F5C6BFA0EF8
:1035E0005D6F5E6BFB0E5F6F606BFD0E616F626BFC
:1035F0006369646B010E656F666F030E676F010E82
:10360000686F050E696F010E6A6F070E6B6F010E12
:103610006C6F080E6D6F010E6E6F0A0E6F6F010EEC
:10362000706F0C0E716F010E726F0E0E736F010EC4
:10363000746F100E756F010E766F120E776F010E9C
:10364000786F140E796F010E7A6F150E7B6F010E75
:103650007C6F170E7D6F010E7E6F190E7F6F010E4E
:10366000806F1B0E816F010E826F1D0E836F010E26
:10367000846F1F0E856F010E866F210E876F010EFE
:10368000886F220E896F010E8A6F240E8B6F010ED8
:103690008C6F260E8D6F010E8E6F280E8F6F010EB0
:1036A000906F2A0E916F010E926F2C0E936F010E88
:1036B000946F2E0E956F010E966F2F0E976F010E61
:1036C000986F310E996F010E9A6F330E9B6F010E3A
:1036D0009C6F350E9D6F010E9E6F370E9F6F010E12
:1036E000A06F390EA16F010EA26F3B0EA36F010EEA
:1036F000A46F3C0EA56F010EA66F3E0EA76F010EC4
:10370000A86F400EA96F010EAA6F420EAB6F010E9B
:10371000AC6F440EAD6F010EAE6F460EAF6F010E73
:10372000B06F480EB16F010EB26F490EB36F010E4C
:10373000B46F4B0EB56F010EB66F4D0EB76F010E25
:10374000B86F4F0EB96F010EBA6F650EBD6FBE6BCD
:10375000670EBF6FC06B690EC16FC26B6B0EC36F1C
:10376000C46B6C0EC56FC66B6E0EC76FC86B700EE8
:10377000C96FCA6B720ECB6FCC6B740ECD6FCE6BF4
:10378000760ECF6FD06B780ED16FD26B790ED36F70
:10379000D46B7B0ED56FD66B7D0ED76FD86B7F0E3B
:1037A000D96FDA6B810EDB6FDC6B830EDD6FDE6B46
:1037B000850EDF6FE06B860EE16FE26B880EE36FC4
:1037C000E46B8A0EE56FE66B8C0EE76FE86B8E0E8E
:1037D000E96FEA6B900EEB6FEC6B920EED6FEE6B98
:1037E000930EEF6FF06B950EF16FF26B970EF36F18
:1037F000F46B990EF56FF66B9B0EF76FF86B9D0EE1
:10380000F96FFA6B9F0EFB6FFC6BA00EFD6FFE6BEA
:10381000A20EFF6F0B01006BA40E016F026BA60ED0
:10382000036F046BA80E056F066BAA0E076F086B7B
:10383000AC0E096F0A6BAD0E0B6F0C6BAF0E0D6FFC
:103840000E6BB10E0F6F106BB30E116F126BB50EC6
:10385000136F146BB70E156F166BB90E176F186BCD
:10386000BA0E196F1A6BBC0E1B6F1C6BBE0E1D6F50
:103870001E6BC00E1F6F206BC20E216F226BC40E19
:10388000236F246BC60E256F266BC70E276F286B20
:10389000C90E296F2A6BCB0E2B6F2C6BCD0E2D6FA3
:1038A0002E6BCF0E2F6F306BD10E316F326BD30E6C
:1038B000336F346BD40E356F366BD60E376F386B73
:1038C000D80E396F3A6BDA0E3B6F3C6BDC0E3D6FF6
:1038D0003E6BDE0E3F6F406BE00E416F426BE10EC0
:1038E000436F446BE30E456F466BE50E476F486BC5
:1038F000E70E496F4A6BE90E4B6F4C6BEB0E4D6F49
:103900004E6BED0E4F6F506BEE0E516F526BF00E13
:10391000536F546BF20E556F566BF40E576F586B16
:10392000F60E596F5A6BF80E5B6F5C6BFA0E5D6F9B
:103930005E6BFB0E5F6F606BFD0E616F626B6369A8
:10394000646B010E656F666F030E676F010E686F23
:10395000050E696F010E6A6F070E6B6F010E6C6FBB
:10396000080E6D6F010E6E6F0A0E6F6F010E706F95
:103970000C0E716F010E726F0E0E736F010E746F6D
:10398000100E756F010E766F120E776F010E786F45
:10399000140E796F010E7A6F150E7B6F010E7C6F1E
:1039A000170E7D6F010E7E6F190E7F6F010E806FF7
:1039B0001B0E816F010E826F1D0E836F010E846FCF
:1039C0001F0E856F010E866F210E876F010E886FA7
:1039D000220E896F010E8A6F240E8B6F010E8C6F81
:1039E000260E8D6F010E8E6F280E8F6F010E906F59
:1039F0002A0E916F010E926F2C0E936F010E946F31
:103A00002E0E956F010E966F2F0E976F010E986F09
:103A1000310E996F010E9A6F330E9B6F010E9C6FE2
:103A2000350E9D6F010E9E6F370E9F6F010EA06FBA
:103A3000390EA16F010EA26F3B0EA36F010EA46F92
:103A40003C0EA56F010EA66F3E0EA76F010EA86F6C
:103A5000400EA96F010EAA6F420EAB6F010EAC6F44
:103A6000440EAD6F010EAE6F460EAF6F010EB06F1C
:103A7000480EB16F010EB26F490EB36F010EB46FF5
:103A80004B0EB56F010EB66F4D0EB76F010EB86FCE
:103A90004F0EB96F010EBA6F650EBD6FBE6B670E2C
:103AA000BF6FC06B690EC16FC26B6B0EC36FC46B0F
:103AB0006C0EC56FC66B6E0EC76FC86B700EC96F8C
:103AC000CA6B720ECB6FCC6B740ECD6FCE6B760E55
:103AD000CF6FD06B780ED16FD26B790ED36FD46B62
:103AE0007B0ED56FD66B7D0ED76FD86B7F0ED96FDF
:103AF000DA6B810EDB6FDC6B830EDD6FDE6B850EA8
:103B0000DF6FE06B860EE16FE26B880EE36FE46BB4
:103B10008A0EE56FE66B8C0EE76FE86B8E0EE96F31
:103B2000EA6B900EEB6FEC6B920EED6FEE6B930EFB
:103B3000EF6FF06B950EF16FF26B970EF36FF46B06
:103B4000990EF56FF66B9B0EF76FF86B9D0EF96F84
:103B5000FA6B9F0EFB6FFC6BA00EFD6FFE6BA20E4F
:103B6000FF6F0C01006BA40E016F026BA60E036FBA
:103B7000046BA80E056F066BAA0E076F086BAC0EE0
:103B8000096F0A6BAD0E0B6F0C6BAF0E0D6F0E6BEA
:103B9000B10E0F6F106BB30E116F126BB50E136F6A
:103BA000146BB70E156F166BB90E176F186BBA0E34
:103BB000196F1A6BBC0E1B6F1C6BBE0E1D6F1E6B3C
:103BC000C00E1F6F206BC20E216F226BC40E236FBD
:103BD000246BC60E256F266BC70E276F286BC90E88
:103BE000296F2A6BCB0E2B6F2C6BCD0E2D6F2E6B8E
:103BF000CF0E2F6F306BD10E316F326BD30E336F10
:103C0000346BD40E356F366BD60E376F386BD80EDB
:103C1000396F3A6BDA0E3B6F3C6BDC0E3D6F3E6BDF
:103C2000DE0E3F6F406BE00E416F426BE10E436F63
:103C3000446BE30E456F466BE50E476F486BE70E2E
:103C4000496F4A6BE90E4B6F4C6BEB0E4D6F4E6B31
:103C5000ED0E4F6F506BEE0E516F526BF00E536FB7
:103C6000546BF20E556F566BF40E576F586BF60E81
:103C7000596F5A6BF80E5B6F5C6BFA0E5D6F5E6B83
:103C8000FB0E5F6F606BFD0E616F626B6369646B4F
:103C9000010E656F666F030E676F010E686F050E8C
:103CA000696F010E6A6F070E6B6F010E6C6F080E65
:103CB0006D6F010E6E6F0A0E6F6F010E706F0C0E3E
:103CC000716F010E726F0E0E736F010E746F100E16
:103CD000756F010E766F120E776F010E786F140EEE
:103CE000796F010E7A6F150E7B6F010E7C6F170EC8
:103CF0007D6F010E7E6F190E7F6F010E806F1B0EA0
:103D0000816F010E826F1D0E836F010E846F1F0E77
:103D1000856F010E866F210E876F010E886F220E50
:103D2000896F010E8A6F240E8B6F010E8C6F260E29
:103D30008D6F010E8E6F280E8F6F010E906F2A0E01
:103D4000916F010E926F2C0E936F010E946F2E0ED9
:103D5000956F010E966F2F0E976F010E986F310EB3
:103D6000996F010E9A6F330E9B6F010E9C6F350E8B
:103D70009D6F010E9E6F370E9F6F010EA06F390E63
:103D8000A16F010EA26F3B0EA36F010EA46F3C0E3C
:103D9000A56F010EA66F3E0EA76F010EA86F400E15
:103DA000A96F010EAA6F420EAB6F010EAC6F440EED
:103DB000AD6F010EAE6F460EAF6F010EB06F480EC5
:103DC000B16F010EB26F490EB36F010EB46F4B0E9F
:103DD000B56F010EB66F4D0EB76F010EB86F4F0E77
:0C3DE000B96F010EBA6F00011200FFD78E
:020000040030CA
:0300010006170ED1
:020005008580F4
:060008000FC00FE00F40E5
:00000001FF
